:100000000C9475010C94AD010C94AD010C94AD01F0
:100010000C94AD010C94AD010C94AD010C94AD01A8
:100020000C94AD010C94AD010C9484190C94561AE7
:100030000C9496140C94AD010C94AD010C94AD018C
:100040000C94AD010C94AD010C94AD010C94AD0178
:100050000C94AD010C941E150C94AD010C94AD01E3
:100060000C94AD010C94AD010C94AD010C94AD0158
:100070000C94AD010C94AD010C94AD010C94AD0148
:100080000C94AD010C94AD010C94AD010C94AD0138
:100090000C94AD010C94AD010C94AD010C94AD0128
:1000A0000C94AD010C94AD010C94AD01C503C503D6
:1000B000F103F103590484058405840577041005D0
:1000C00021052105C31AEA1AE21BEA1AE21B361BB4
:1000D000591BE21BB01BBF1B29001E001F00200084
:1000E00021002200230024002500260027002D00E7
:1000F0002E0031002A002B0014001A000800150001
:1001000017001C0018000C00120013002F00300014
:1001100031000000390004001600070009000A0041
:100120000B000D000E000F003300340031002800DA
:100130000000E10064001D001B000600190005001E
:1001400011001000360037003800E5005241000071
:10015000E000E300E2000000000000002C000000CE
:1001600000000000E600E7006541E4000000010037
:100170000100010001000100010001000100010077
:100180000100010001000100010001000100010067
:100190000100010001000100010001000100010057
:1001A000010001000100005C0000010001000100ED
:1001B0000100010001000100010001000100010037
:1001C0000100010001000000010001000100010028
:1001D0000100010001000100010001000100010017
:1001E000010001000000010001000100000000000A
:1001F00000000100000000000000010001000100FB
:1002000001000000100350006C00610069006E00E6
:100210003600300000000E034500760079006400CF
:100220003100330000000403090409023B0002010D
:1002300000A0FA09040000010301010009211101D5
:1002400000012240000705810308000109040100A4
:1002500001030000000921110100012232000705FD
:10026000820320000112010002000000080547601F
:100270000101000102000105010980A101850319A6
:10028000012AB700150126B700950175108100C03D
:10029000050C0901A101850419012AA002150126F6
:1002A000A002950175108100C005010906A1010594
:1002B0000719E029E71500250195087501810295C8
:1002C00001750881010507190029FF150026FF00A7
:1002D0009506750881000508190129059505750120
:1002E0009102950175039101C00011241FBECFEF4B
:1002F000DAE0DEBFCDBF04B603FE18C0809168020D
:1003000090916902A0916A02B0916B028730904B84
:10031000A740B04B59F410926802109269021092F3
:100320006A0210926B02E0E0F8E3099511E0A0E0A8
:10033000B1E0EAEDF8E302C005900D92A838B107EC
:10034000D9F722E0A8E8B1E001C01D92A836B207B3
:10035000E1F70E9476110C946B1C0C94000081E074
:10036000089581E008950C94B10108950C94B501AD
:100370001F93CF93DF9300D000D01F92CDB7DEB78D
:1003800049835A836B8330918B0189819A81311122
:1003900014C0662359F0222349F00E94BD07182F8C
:1003A000682F89819A810E94660703C00E94910785
:1003B000182F69817A81812F04C00E94BD0769814D
:1003C0007A810F900F900F900F900F90DF91CF9147
:1003D0001F910C94E10EFC01262F40815181628116
:1003E000738184810C94B80181E00895CF93DF93E9
:1003F000EC0160E00E94EB01BE01DF91CF910C9413
:10040000B6010C9427100C94231008950E94100636
:100410000E9405022FEF84E39CE021508040904031
:10042000E1F700C000000C9444150F931F93CF9385
:10043000DF938C0161E00E94EB01EC01B8010E94A6
:10044000B3018823F1F1B801CE010E946F13882314
:10045000C1F1B801CE010E948311882391F1B80146
:10046000CE010E94CB12882361F1F801828188239A
:1004700009F1CB358DE5D807C1F050F4C115FCE585
:10048000DF0781F0CF3DDC45A9F40E94F40C19C0D0
:10049000CC35EDE5DE0761F0CD35DD4559F40E9440
:1004A000370C08C00E9406020CC00E94400C02C01B
:1004B0000E94430CC801DF91CF911F910F910C94C2
:1004C000AF0180E0DF91CF911F910F9108950E94BD
:1004D00078140C9480020E9483020C947E14089578
:1004E0000C946F0281E008950C9472020895CF93EA
:1004F000C82F0E9470028C2F0E947402CF91089521
:1005000080E00C9477020E94CB130C9477020E9437
:10051000CB1390918A01891721F080938A010C9462
:1005200077020895CF93DF93CDB7DEB72B970FB641
:10053000F894DEBF0FBECDBF4F83588769877A8797
:100540008B8761110E94830B9E012F5F3F4F86E0D6
:10055000F90111928A95E9F785E0FE013796D901F4
:1005600001900D928A95E1F789819A814C815D8194
:10057000452B31F09F3F31F491E08F3F19F403C0D8
:1005800091E001C090E090FF09C049815A816B81E0
:100590007C818D819E810E94A40A05C0C9010E94B0
:1005A000F4018111F2CF2B960FB6F894DEBF0FBE87
:1005B000CDBFDF91CF910895FC01808191810E9490
:1005C000FF070895CF93882309F448C0C82F8CEF04
:1005D0008C0F813AD0F46C2F80910201909103012D
:1005E0000E941A14882349F06C2F80910201909187
:1005F00003010E9452140E94A50B6C2F80910201EE
:10060000909103010E9450140CC080E28C0F88303E
:1006100058F4C77081E001C0880FCA95EAF70E94BC
:10062000660BCF910C94A50BEBE5EC0FE33040F497
:10063000F0E0E15CFE4F808190E0CF910C94E213FA
:10064000C85AC73158F4EC2FF0E0EE0FFF1FEF5EF1
:10065000FE4F80819181CF910C94F813CF91089532
:10066000882349F1682F8CEF860F813A38F4809106
:100670000201909103010E9452140CC080E2860F87
:10068000883050F4677081E001C0880F6A95EAF7FE
:100690000E946C0B0C94A50B8BE5860F833020F425
:1006A00080E090E00C94E213685A673120F480E017
:1006B00090E00C94F81308951F93CF93DF93182FB5
:1006C000EB010E94E202209741F08FE99FE0019741
:1006D000F1F700C000002197F6CF812FDF91CF9175
:1006E0001F910C943003893319F060E070E002C070
:1006F00060E570E00C945C03882321F00E94660B97
:100700000C94A50B0895882321F00E946C0B0C9487
:10071000A50B0895CF92DF92EF92FF920F931F9354
:10072000CF93DF937C01D62FC72FFC011281058167
:1007300002950F700E945C0B8823B9F01123A9F079
:100740008C2F807F803421F080E28D0F883068F01C
:100750008091420282FD09C082E00E94050C0E9445
:100760005C0B91E0D82ED92601C0D12CCC2EC2949E
:100770008FE0C8228C2D90E08C30910508F0C4C128
:10078000FC01EA5AFF4F0C94161C8C2F807FCF700F
:10079000882311F0C295C07F112399F0CC2309F46E
:1007A0009FC180E28D0F883010F0D11104C08C2FD2
:1007B0000E94660B03C08C2F0E94760B0E94A50B33
:1007C0008FC18D2F0E943003CC2309F49DC180E29C
:1007D0008D0F883038F1DD2329F18C2F0E947C0B9E
:1007E00024C08C2F807FCF70803211F0C295C07FE3
:1007F000DD2319F0D130A1F13DC08091420282FF8A
:1008000017C0112349F0CC2329F08C2F0E94660BCE
:100810000E94A50B80E065C180E00E943003CC23DC
:1008200009F472C18C2F0E946C0B0E94A50B6CC145
:10083000112371F0002341F0013031F40E94860B46
:100840008C2B0E948E0B60C10E94860B8C2B1DC0CE
:10085000002319F0013009F457C10E949B0B25C0F9
:10086000112321F0063008F04FC10EC0053008F00A
:100870004BC11BC0112361F0002331F0F7018581CA
:1008800080FF2EC18F7085838C2F0E947C033CC11A
:10089000002359F0D93309F034C1FFEF07EE13E01C
:1008A000F15000401040E1F72AC18C2F0E948303D1
:1008B0002BC18C2F86958695837019F0813061F05D
:1008C00023C1112321F08D2F9C2F937002C080E053
:1008D00090E00E94E21320C1112321F08D2F9C2F64
:1008E000937002C080E090E00E94F81315C18C2F35
:1008F000837009F047C011110BC12D2F2295269549
:100900002770220F220F6D2F6F70862F90E0A0E0CE
:10091000B0E0022E04C0880F991FAA1FBB1F0A94C3
:10092000D2F7D4FF10C04FE050E060E070E004C0A8
:10093000440F551F661F771F2A95D2F74095509593
:100940006095709503C040E050E0BA01C695C69529
:10095000C3708A019B01082B192B2A2B3B2BC90141
:10096000B801C23049F058F4C13019F00E947C0639
:10097000CFC00E946A06CCC00E948E06C9C00E94E9
:100980006806C6C0112319F08C2F817001C08695AE
:10099000882309F4BDC02D2F229526952770220F9C
:1009A000220F6D2F6F70862F90E0A0E0B0E0022E36
:1009B00004C0880F991FAA1FBB1F0A94D2F7D4FF47
:1009C00010C04FE050E060E070E004C0440F551FDD
:1009D000661F771F2A95D2F74095509560957095C0
:1009E00003C040E050E0BA01C695C695C3708A01C5
:1009F0009B01082B192B2A2B3B2BC901B801C230B4
:100A000049F058F4C13019F00E94410781C00E949A
:100A10002F077EC00E9453077BC00E94A20678C0A9
:100A2000CF70112339F08C2F0E94C8068D2F0E94A1
:100A30007C036EC08D2F0E9483038C2F0E94E906D9
:100A400067C0D23F21F128F4D03F41F0D13FC1F03F
:100A500043C0D33F19F1D43F79F03EC0112341F098
:100A6000053008F051C08C2F8F710E940E074CC0CA
:100A7000063008F049C0F7CF8091420282FF18C0CB
:100A8000112339F08C2F8F710E94C8063DC01123AD
:100A9000C9F38C2F8F710E94E90636C0112329F00B
:100AA0008C2F8F710E94B3062FC00E94AE062CC0FF
:100AB000112349F0CF718C2F0E94C80663E08C2F60
:100AC0000E94EA0B21C081E00E94050C0230E0F098
:100AD00082E00E94050C18C0112331F0002391F22E
:100AE0008D2F0E94E20210C0002399F2D93349F4FD
:100AF0001FEF27EE33E0115020403040E1F700C0F7
:100B000000008D2F0E94300388EF8C0D843020F47C
:100B10000E94CB130E947702DD20C9F00E94580B7F
:100B200080FD15C0F70112820E94520B0E94C80678
:100B3000C7010E94C8050E94520BDF91CF911F91FF
:100B40000F91FF90EF90DF90CF900C94E906DF912A
:100B5000CF911F910F91FF90EF90DF90CF9008956C
:100B60000F931F93CF93DF93EC01688179818A8182
:100B70000E940A088C010E9465070E945606B8016F
:100B8000CE010E948A03DF91CF911F910F910895AA
:100B9000CF93DF93EC01988189812B813C81232BBA
:100BA00031F08F3F31F481E09F3F19F403C081E0C1
:100BB00001C080E080FD1DC0CE010E9415028111A0
:100BC00010C00E945C0B8823A1F08A81882389F0E1
:100BD0008091420282FD0DC082E0DF91CF910C94A2
:100BE000050CCE010E94B005CE01DF91CF910C948F
:100BF000F601DF91CF91089580E090E00E94E2132A
:100C000080E090E00E94F8130E94830B0C94A50BE7
:100C100080910201909103010E9454140C94FC05F0
:100C20000E94730B0C94080692959F70963079F091
:100C300010F4925001C09A50923068F4803F69F0ED
:100C400018F4883E40F409C0843F29F406C0883E69
:100C500020F0813F11F080E0089581E00895FC01CB
:100C6000808191810E94FF070E9414060895CF930E
:100C7000DF9300D000D01F92CDB7DEB70F900F905A
:100C80000F900F900F90DF91CF910895CF93DF9346
:100C900000D000D000D0CDB7DEB726960FB6F894BE
:100CA000DEBF0FBECDBFDF91CF91089508950895A7
:100CB0000C9457060C9458060E945A066093C20181
:100CC0007093C3018093C4019093C5010C94FC05FB
:100CD0000C945C060F931F930091C2011091C30105
:100CE0002091C4013091C501602B712B822B932B75
:100CF0001F910F910C945C060F931F930091C201FA
:100D00001091C3012091C4013091C501602371236A
:100D1000822393231F910F910C945C060F931F93D2
:100D20000091C2011091C3012091C4013091C5010D
:100D300060277127822793271F910F910C945C06DF
:100D40000C9457060E94A0066093BE017093BF01E9
:100D50008093C0019093C1010C94FC0560E070E0A9
:100D6000CB010C94A2060F931F9341E050E060E08A
:100D700070E08A019B0104C0000F111F221F331F66
:100D80008A95D2F7C901B8011F910F910C94A20660
:100D90000F931F9341E050E060E070E004C0440F07
:100DA000551F661F771F8A95D2F78091BE019091DB
:100DB000BF01A091C001B091C1018A019B01082B24
:100DC000192B2A2B3B2BC901B8011F910F910C94B1
:100DD000A2060F931F9341E050E060E070E004C072
:100DE000440F551F661F771F8A95D2F7409550957F
:100DF000609570958091BE019091BF01A091C00156
:100E0000B091C1018A019B01082319232A233B23A6
:100E1000C901B8011F910F910C94A2060F931F9363
:100E200041E050E060E070E004C0440F551F661FD1
:100E3000771F8A95D2F78091BE019091BF01A09152
:100E4000C001B091C1018A019B01082719272A27F7
:100E50003B27C901B8011F910F910C94A2060F9373
:100E60001F930091BE011091BF012091C0013091EC
:100E7000C101602B712B822B932B1F910F910C942E
:100E8000A2060F931F930091BE011091BF01209104
:100E9000C0013091C10160237123822393231F91EC
:100EA0000F910C94A2060F931F930091BE01109115
:100EB000BF012091C0013091C101602771278227B5
:100EC00093271F910F910C94A20608952FE0929FF3
:100ED000800D1124E82FE695E695E695877051E0A0
:100EE00001C0550F8A95EAF785E0E89FF0011124CB
:100EF000E457FE4F20E030E070E04081CB01022E4D
:100F000002C0969587950A94E2F7817081958427AF
:100F10008523842781932F5F3F4F2530310569F763
:100F200008952FE0929F800D1124682F6695669595
:100F30006695982F977085E0689FB001112440E076
:100F400050E080E0FB01E40FF51FE457FE4F2081E5
:100F500030E0092E02C0369527950A94E2F72170F9
:100F60003327042E01C0220F0A94EAF7822B4F5F29
:100F70005F4F4530510531F70895BF92CF92DF9210
:100F8000EF92FF920F931F93CF93DF938C01C0904A
:100F9000BE01D090BF01E090C001F090C1018091EE
:100FA000C2019091C301A091C401B091C501C82AAA
:100FB000D92AEA2AFB2ACFE1D0E0D701C6010C2EBC
:100FC00004C0B695A795979587950A94D2F780FDAA
:100FD00004C0219790F7B12C07C0BC2EB8018C2F0C
:100FE0000E94F40E0197A9F38B2DDF91CF911F91F1
:100FF0000F91FF90EF90DF90CF90BF900895CF9327
:10100000DF93EC010E94BD07BE010E94F40EDF9148
:10101000CF9108951F93CF93DF93EB0190918B01B4
:10102000992321F0CB010E94FF0713C0882349F0C8
:10103000CB010E94BD07182F682FCE010E946607C2
:1010400004C0CB010E949107182FBE01812F0E947E
:10105000F40EDF91CF911F9108951F93CF93DF93EB
:10106000C091C60116E08091C701C81799F0D0E081
:101070001C9FF0011D9FF00D1124E853FE4F40818D
:10108000518162817381848195810E9446062196F7
:10109000C770E9CFDF91CF911F9108954091F8017A
:1010A0005091F9016091FA017091FB018091FC016E
:1010B0009091FD010C944606EF92FF920F931F93BF
:1010C000CF93DF938091FD0182958F7009F065C009
:1010D0008091FA01882309F460C08091C601F090E4
:1010E000C7011091F8010091F9016091FB01709125
:1010F000FC0191E01F3F09F090E0C0910001D09108
:101100000101292F96E0E92E8F1509F446C06115DB
:10111000710521F00F3F21F030E003C031E001C044
:10112000322F90E030FD36C0E89EF001E99EF00DD0
:101130001124DF01A853BE4F11963C911197301333
:1011400029C03C91311326C012963C91129731115F
:1011500021C013964D915C911497461B570B4C1769
:101160005D07C0F48091FD018F7080618093FD0167
:10117000E353FE4F80818F708061808388EF91E020
:101180000E94C805DF91CF911F910F91FF90EF90C2
:101190000C942D0801968770B7CFDF91CF911F91E6
:1011A0000F91FF90EF9008959F92AF92BF92CF92D0
:1011B000DF92EF92FF920F931F93CF93DF93CDB700
:1011C000DEB761970FB6F894DEBF0FBECDBF8C01BE
:1011D00085E0F801DE011D9601900D928A95E1F7F8
:1011E000D8011296EC909091F801E091F9012091CC
:1011F000FB013091FC012115310531F0EF3F31F455
:1012000081E09F3F19F403C081E001C080E0B82F66
:10121000B1709B2E80FD47C1D8014C9111965C9115
:1012200011971396AD90BC90149788EFC82E81E06B
:10123000D82EF090FA01B501621B730B20910001CA
:1012400030910101FF2009F4D9C08091FD0162179E
:10125000730708F095C0282F207F09F052C05E1355
:1012600013C0491311C0FE2CE1100EC08F708061B5
:101270008093FD010E944E08C6010E94C80580911E
:10128000FD01F80185834DC1AB2831F05F3F31F49A
:1012900081E04F3F19F403C081E001C080E080FD90
:1012A00003C081E08E2502C080E090E0F82FF1704D
:1012B000FF2E80FF1CC08091C6012091C70136E03F
:1012C000821709F40BC190E0389FF001399FF00DAF
:1012D0001124E853FE4F6181561306C06081461306
:1012E00003C06281E61203C001968770E9CFFE2C2D
:1012F000EE2009F416C18091FD0181608093FD010B
:1013000054C05E1306C0491304C0E11002C0F801C6
:1013100099C0C8010E942F06882361F1EE2051F187
:101320002091FD01822F82958F7090E0029774F0DA
:101330008091F8019091F90198878F831986BB8677
:10134000AA862C87CE0107960E94C80586E0F80180
:10135000A8EFB1E001900D928A95E1F70E945C0838
:101360000E944E080AC05E1711F1C8010E942F06A4
:1013700081112CC0C8010E94C805FF24F394D1C07C
:10138000282F207F81F77A2DB98AA88A6E2D898926
:101390000E94370688EF91E00E94C80586E0D601DA
:1013A0001D928A95E9F70E944E08F12CBAC04913A4
:1013B000DCCFE110DACFF8018583C8010E94C805AF
:1013C00086E0D6011D928A95E9F7ABC0EE2091F236
:1013D0002091FD01822F82958F7090E002970CF48E
:1013E000B5CF8091F8019091F9019A8389831B828E
:1013F000BD82AC822E83CE010196A6CF6217730701
:1014000008F044C0FE2CEE2009F4B4CF5E1330C0C7
:1014100049132EC02091FD0120FD21C0822F82950D
:101420008F70482F50E041155105C9F0F801258310
:101430004F30510541F08F5F982F9295907F822F0A
:101440008F70892B8583C8010E94C80586E0F8014A
:10145000A8EFB1E001900D928A95E1F73CC086E0DB
:10146000F801A8EFB1E001900D928A95E1F759C01B
:10147000C8010E942F06811169CF8091FD01816012
:101480008093FD01C8010E94C8054BC07A2DB98A1E
:10149000A88A6E2D89890E94370686E0D6011D92A2
:1014A0008A95E9F718C0EE2009F464CFC8010E94BC
:1014B0002F06F82E882309F45DCF86E0F801A8EF07
:1014C000B1E001900D928A95E1F788EF91E00E94DA
:1014D000DC020E945C080E944E0823C04D875E8794
:1014E0008D859E850E94FF07292F22952F7022301F
:1014F00028F49F7039F0811105C00BC0243028F406
:101500009F7049F4805E883020F0C8010E94C805B1
:101510009F2CF92C06C0D80115969C91907F91F7CD
:10152000F8CF8F2D61960FB6F894DEBF0FBECDBFFA
:10153000DF91CF911F910F91FF90EF90DF90CF90AF
:10154000BF90AF909F9008951F93CF93DF93CDB737
:10155000DEB72C970FB6F894DEBF0FBECDBF4F831A
:10156000588769877A878B879C87CE0107960E9468
:10157000D4088823D1F09F8188852A853B85232B39
:1015800031F08F3F31F481E09F3F19F403C081E0D7
:1015900001C080E080FD47C04F81588569857A850C
:1015A0008B859C850E9446063EC086E0FE013796EC
:1015B000DE01119601900D928A95E1F7FF81E88591
:1015C0006A857B856115710531F0EF3F31F481E06B
:1015D000FF3F19F403C081E001C080E080FD23C01B
:1015E0002091C70130E0C901019687709927409189
:1015F000C60150E084179507F1F1F983EA837D83F2
:101600006C8396E0929FD001939FB00D1124A85354
:10161000BE4FFE01319601900D929A95E1F78093AD
:10162000C7010E942D0816E08091C6019091C70164
:10163000891771F1189FC001112488539E4F0E9491
:10164000D408882329F1E091C6011E9FF0011124DE
:10165000E853FE4F4081518162817381848195817D
:101660000E9446068091C60190E0019687709927F6
:101670008093C601D9CF0E9410061092C701109224
:10168000C601E8EFF1E086E0DF011D928A95E9F7F7
:101690002C960FB6F894DEBF0FBECDBFDF91CF9171
:1016A0001F910895809106028595859585950895E9
:1016B000809106028770089590910602977081E0EC
:1016C00009F480E00895809111020895909111022B
:1016D000892B80931102089580959091110289239E
:1016E00080931102089510921102089590911002B2
:1016F000892B809310020895809590911002892380
:1017000080931002089510921002089580910702AC
:10171000089508950C94890B0C948A0B90914202C1
:1017200092FD08C090910702981721F0809307025C
:101730000C948C0B089580910702882329F0109255
:10174000070280E00C948C0B0895CF93DF93E09117
:101750000201F0910301809111028083E091020166
:10176000F0910301908180911002892B80838091F8
:101770000702882381F0E0910201F091030190813A
:10178000892B808380910201909103010E940E14A5
:1017900081110E949B0BC0910201D091030148E08E
:1017A00050E06EEF71E0CE010E941C1C892B69F0A5
:1017B00088E0FE01AEEFB1E001900D928A95E1F76D
:1017C000CE01DF91CF910C94D713DF91CF91089583
:1017D0000C94890B9091420292FD10C098E0899F71
:1017E00090011124262B209306020E94C8068091A6
:1017F00006028595859585950C94E80B0C94C80692
:101800001092060280E00C94E80B2091060280956D
:10181000822380930602982F977099F430E0482F26
:10182000082E000C550B2417350759F090914202F1
:1018300092FD07C08595859585950E94E9060C94D3
:10184000000C08959091420292FB222720F928175C
:1018500069F080FB92F9909342028091410290914D
:1018600042020E94700C82E00C94050C0895809155
:10187000420282FB882780F991E089270C94220C90
:1018800081E00C94220C80E00C94220C6FEF7FEF2F
:1018900080E090E00C94551C80E090E00E94311CA8
:1018A00021E0893E9E4F09F020E0822F089582E0DA
:1018B00090E00C94291C83E090E00C94291CCF93B9
:1018C00084E090E00E94291CC82F82E290E00E94F0
:1018D000291C2C2F30E0A901582BCA01CF91089563
:1018E000CF93C92F682F84E090E00E94371C6C2FA3
:1018F00082E290E0CF910C94371CAB01BC018FE0E9
:1019000090E00C94491CAB01BC0183E190E00C9485
:10191000491C60E070E0CB010C94830C60E070E047
:10192000CB010E947D0C0C94890C69EE7EEF80E067
:1019300090E00E94551C60E082E090E00E94371C1D
:1019400060E083E090E00E94371C1092C201109288
:10195000C3011092C4011092C50160E084E090E0E0
:101960000E94371C60E082E290E00E94371C60E039
:1019700085E090E00E94371C60E086E090E00E94E5
:10198000371C6FEF87E090E00E94371C40E050E08A
:10199000BA0188E090E00E94491C60E08DE090E090
:1019A0000E94371C40E050E0BA0188E190E00E94BC
:1019B000491C60E087E190E00E94371C40E050E065
:1019C000BA018CE190E00E94491C60E070E080E286
:1019D00090E00E94551C40E050E0BA0188E190E0A0
:1019E0000E94491C0C948E0C0C94950C682F8EE070
:1019F00090E00C94371C0E940315609320027093B2
:101A00002102809322029093230260931C02709320
:101A10001D0280931E0290931F02089585B780686F
:101A200085BF85B7806885BF089581E008950C94CF
:101A3000150D08950C94190D0C94190D0C941C0D92
:101A40000C94190D0C94200D0C94190D0E940E0D80
:101A500080ED9FE00E94C1130E94240D0C94220D82
:101A60000E941A0D0C94190D0E94EA0F0C94760234
:101A70000E94EE140E94CF100E94340D0C941E0D93
:101A80005F926F927F928F929F92AF92BF92CF920E
:101A9000DF92EF92FF920F931F93CF93DF93CDB717
:101AA000DEB72A970FB6F894DEBF0FBECDBF0E94F7
:101AB000E410C82E81110E94FB0C32E1832E32E02B
:101AC000932E00E010E0502E802F0E940E105C013B
:101AD000F401619071904F016826792661147104B8
:101AE000B1F40F5F1F4F0530110569F78FEF898340
:101AF0008A831B820E94F7148160782F9D838C83D8
:101B000049815A816B818D810E9492023AC08091F5
:101B1000240281FD0E941710D12CEE24E394F12CB5
:101B2000C3018E219F21892B29F10E94170D882343
:101B3000A9F0DE825F82AE20BF2081E0AB2809F4ED
:101B400080E088870E94F7148160782F9A878987C0
:101B50004E815F8168858A850E949202000F111F65
:101B6000F801EE5EFD4F80819181E826F926F18231
:101B7000E08207C0D394EE0CFF1CFFE0DF12D0CF51
:101B8000B0CF81E0C11001C080E02A960FB6F89472
:101B9000DEBF0FBECDBFDF91CF911F910F91FF90A0
:101BA000EF90DF90CF90BF90AF909F908F907F90FD
:101BB0006F905F9008950E94400D0C948702CF9320
:101BC000DF930E94F90EEC01811522E59207E8F5FA
:101BD000811531E5930708F0B6C0883E910528F5D8
:101BE000803E910508F0E9C0883A910570F4853A85
:101BF000910508F07AC08130910509F473C008F4AA
:101C0000D9C0049708F0D9C0D5C08F3B910508F022
:101C1000D1C0C85AD0E0CC0FDD1FCE5BDE4F09909B
:101C2000D881C02DCE019464C9C0811540E59407C8
:101C300008F069C0811550E4950708F060C09A95D6
:101C400081159F4108F4B9C0B5C0811536E59307E9
:101C500028F5811545E5940708F092C0811554E5F3
:101C6000950708F087C0AC0143705527282F2695AB
:101C70002695C115D34508F06CC081E090E002C004
:101C8000880F991F4A95E2F740E2249F90011124A2
:101C9000EC01C22BD32BCE019C6890C081152AE5A4
:101CA000920780F4811539E5930708F072C0811519
:101CB00048E5940708F47EC0D82FCC27CE01806F6A
:101CC000906A7CC090568115904208F073C08D2FA9
:101CD0008F710E948D0FDD27D0628F71AE01582B5E
:101CE000CA016CC081E090E069C0C55AD0E0C0591B
:101CF000DE4F8881C82FD0E0CE0190645FC0DF70D6
:101D0000CE01906A5BC074E0969587957A95E1F76D
:101D1000282F23703C2F337081E090E002C0880FA1
:101D2000991F3A95E2F79C68AC01522B9A019C2FBF
:101D30009F709695969550E2959FE0011124C901F8
:101D40008C2B9D2B3BC0D82FCC27CE01816F906A66
:101D500035C081E090E002C0880F991F4A95E2F7F4
:101D600050E2259F90011124EC01C22BD32BCE0110
:101D70009A6824C0D82FCC27CE01846F906A1EC0E9
:101D80000E948D0F8F7190E0D82FCC27CE019062EA
:101D900015C08F700E948D0F94E0D695C7959A95C7
:101DA000E1F7CF70D0E0DC2FCC27D0699E01282B43
:101DB000C90104C080E090E001C0CE01DF91CF9165
:101DC00008952BE4829FC0011124FC012FE0729F33
:101DD000E00DF11D1124E60FF11DEE0FFF1FE8527B
:101DE000FF4F8591949108950E94E10E0E94DF0DAE
:101DF00008958238910569F1B0F48133910509F4B1
:101E00006DC048F48932910509F463C08A329105A6
:101E100009F469C008958533910509F455C08933E3
:101E20009105B9F00895833E910569F138F4803E3B
:101E30009105B1F0823E910509F10895863E910524
:101E4000A9F1873E9105B9F1843E910509F064C07E
:101E500023C02091410220FD4FC021FD4DC00895B7
:101E60008091410280FD44C08091420280FF44C0C5
:101E70008091410284FD42C083EE4DC080914102B9
:101E800082FF38C0F5CF8091410282FD33C080913E
:101E9000420280FD31C0ECCF8091420281FF32C00E
:101EA0008091410284FD2AC087EE35C080914102B5
:101EB00083FF26C0F5CF8091410283FD21C0809130
:101EC000420281FD1FC0ECCF8091410285FD1CC004
:101ED0001DC08091410285FD19C016C0809141024C
:101EE00086FD16C017C08091410286FD13C010C048
:101EF00089E311C082EE0FC080EE0DC080E00BC000
:101F000086EE09C084EE07C089E205C085E303C000
:101F10008AE201C081E390E008959091410292FF2E
:101F20000DC0282F2871283019F4877F846006C0DF
:101F3000282F2471243011F48B7F886093FF0DC00B
:101F4000282F2871283119F4877E846106C0282F34
:101F50002471243111F48B7E88612091420220FF8C
:101F60000DC0382F3871383019F4877F816006C072
:101F7000382F3171313011F48E7F886021FF0DC010
:101F8000282F2871283119F4877E816106C0282FF7
:101F90002171213111F48E7E886194FD877E089530
:101FA00080E008950C94460C0E94E4108FE39CE9B5
:101FB0000197F1F700C000000E94E41080E00E9449
:101FC0000E1080FF04C00E94D20F0C944415089597
:101FD0000C94D40F0E944C0C811102C00E94F40C8E
:101FE0000E94570C809324020E945F0C909342023F
:101FF000809341020E94E80F0E945B0C682F70E002
:1020000080E090E00E9468066091BE017091BF017F
:102010008091C0019091C1010C94A006E82FF0E0DE
:10202000EE0FFF1FE35BFD4F8081918108950895BE
:1020300080EA8A95F1F7089500C008950C9418106D
:1020400008950C9420100C9421100C9420100C94E2
:102050002510F894E82FE295EF70F0E031A1282FD9
:102060002F7081E090E001C0880F2A95EAF7982F41
:102070009095932391A392A1892B82A3789408959C
:102080000F931F93CF93DF93C2E8D1E089918F3FE5
:1020900011F00E94291081E0C738D807B9F7C3E7CB
:1020A000D1E002E811E089918F3F11F00E942910E0
:1020B0000C171D07C1F7DF91CF911F910F91089564
:1020C000BF92CF92DF92EF92FF920F931F93CF9325
:1020D000DF938C01C62FD0E0CE018E579E4F6C014E
:1020E000FC0190819F3F09F450C0B62EF894E92F6F
:1020F000E295EF70F0E081A19F7021E030E001C037
:10210000220F9A95EAF7822B81A382A1209528239A
:1021100022A378940E941C10E3E7F1E042E851E02A
:1021200021E030E0E12CF12C61916F3F89F0A62F86
:10213000A295AF70B0E090968C9190E06F7002C065
:10214000959587956A95E2F780FD02C0C90102C0A6
:1021500080E090E0E82AF92A220F331F4E175F072C
:1021600019F7F60180818F3F11F00E94291061E07C
:10217000E114F10409F460E08B2D0E941E10CC0FD5
:10218000DD1FC00FD11FF982E882DF91CF911F912F
:102190000F91FF90EF90DF90CF90BF9008950E9435
:1021A00040108AE0EDE4F2E0DF01982F1D929A954D
:1021B000E9F7E3E4F2E0DF011D928A95E9F785E0B3
:1021C0000E942F110C940102FF920F931F93CF9343
:1021D000DF93CDB7DEB72A970FB6F894DEBF0FBEF8
:1021E000CDBF8E010F5F1F4F8AE0F80111928A95D3
:1021F000E9F7F12C6F2DC8010E946010F394F5E00F
:10220000FF12F8CF4AE050E0B80183E492E00E9468
:102210001C1CFF24F394009709F4F12C892B41F046
:102220008AE0F801A3E4B2E001900D928A95E1F70B
:102230002F2D45E06DE472E083E492E00E943011BE
:102240000E9403028F2D2A960FB6F894DEBF0FBEB0
:10225000CDBFDF91CF911F910F91FF900895089509
:10226000FF920F931F93CF93DF93F82E092F162F12
:10227000D72FC42F222349F081E0809327020E94A8
:10228000F7149093260280932502809127028823D9
:10229000D9F080912502909126020E940F15059792
:1022A00098F0EF2DF02FA12FBD2F80E090E04C2F64
:1022B00050E08417950734F4219131912D933D938B
:1022C0000196F7CF10922702DF91CF911F910F91C6
:1022D000FF9008950E94DC160E94380D0C94E816B9
:1022E0000E94EC160E94DB0D0C9406170E949514B8
:1022F0000E94C3160E94260D0E946A110E9470114E
:102300000E94300DFBCFCF93DF93EC01FB01828164
:10231000882309F43CC1C430FDE5DF0760F4CB3FFE
:102320009CE5D90788F49E0122503C4524313105B3
:1023300008F02EC109C0C236EDE5DE0729F0C63A25
:10234000FDE5DF0709F024C10E945F0C9093420273
:1023500080934102C1318CE5D80709F4C6C008F06A
:1023600042C0C930ECE5DE0709F49BC000F5C5307A
:102370008CE5D80709F485C078F4C330ECE5DE07B6
:1023800009F478C008F07AC0C230DC4509F0F5C025
:10239000809141028160EFC0C7309CE5D90709F404
:1023A00078C008F07AC0809141028061E4C0CD30ED
:1023B000FCE5DF0709F487C058F4CB309CE5D9076A
:1023C00009F479C008F07BC08091410288606FC039
:1023D000CF30FCE5DF0709F480C008F082C08091AF
:1023E0004102877FC8C0CE3F9CE5D90709F471C080
:1023F00000F5C531FCE5DF0709F485C068F4C33199
:102400009CE5D90709F475C008F095C00E94100634
:10241000809141028F77AFC0CC3FFCE5DF07A9F187
:1024200008F054C0CB3FDC4509F0A7C080914202C0
:1024300040C0C230EDE5DE0709F489C058F4C1158B
:102440008DE5D80709F45AC008F069C080914202AE
:1024500082602FC0C236EDE5DE0709F47CC0C63AC3
:10246000FDE5DF0709F481C0C330DD4509F085C013
:1024700080E06EC08091410282607DC08091410207
:1024800016C080914102886076C0809142028260CD
:102490004FC08091410280626EC080914102806491
:1024A0006AC00E94100680914102806864C0846006
:1024B00062C081603DC0809141028E7F5CC080918E
:1024C00041028D7F58C08091410216C08091420226
:1024D00018C0809142028D7F2BC0809141028F7E77
:1024E0004AC0809141028F7D46C0809141028F7B1E
:1024F00042C080914102877F8B7F3DC08091420224
:102500008D7F8E7F15C08091410282FB222720F9AA
:1025100091E0922790FB82F990FB83F92CC0809187
:102520004202982F909591708E7F892B90FB81F9B4
:102530008093420222C00E9410068091410287FBD4
:10254000222720F991E0922790FB87F914C081E0BF
:102550000E94F60C12C08091410284FB222720F9D0
:1025600091E0922790FB84F906C080914102982F58
:10257000909590FB80F98093410280914102909167
:1025800042020E94700C0E94100680E001C081E0AF
:10259000DF91CF910895CF93DF9386319C4541F52C
:1025A000EB010E94630B982F8A81209102013091E8
:1025B0000301882379F09A7A81E009F480E080931E
:1025C0002802911102C069E201C065E3C9010E94BD
:1025D00050140AC080912802811102C069E201C032
:1025E00065E3C9010E9452140E94A50B80E001C05E
:1025F00081E0DF91CF9108950F931F93CF93DF93E5
:10260000C42FD22FFC0182818823C9F040932B0272
:102610000E94F71490932A028093290280E28C0F83
:10262000883008F057C0C77081E001C0880FCA9594
:10263000EAF7DF91CF911F910F910C947C03809169
:102640002B02481330C08091290290912A020E94E7
:102650000F15883C910538F510E21D0FCD17B9F024
:1026600080E28C0F883040F4C77081E001C0880F91
:10267000CA95EAF70E948303183028F581E09D2F60
:10268000977001C0880F9A95EAF70E947C03802F0B
:102690000E9473031830F0F4D77081E001C0880FF6
:1026A000DA95EAF70AC080E28C0F883098F4C77098
:1026B00081E001C0880FCA95EAF7DF91CF911F91A1
:1026C0000F910C948303802FDF91CF911F910F9175
:1026D0000C947303DF91CF911F910F9108950F9385
:1026E0009C01CB01243F4CE5340731F188F4293DAE
:1026F000FCE53F07D9F02A3D4CE5340779F1283D48
:102700003C45A9F506E221EE41EE68ED7CE52BC0E3
:10271000263FFCE53F07E1F0A8F0273F3C4539F5AF
:1027200007E225EE46EE67EF7CE51DC007E225EEE9
:1027300045EE69ED7CE517C006E221EE40EE64EF60
:102740007CE511C007E225EE44EE65EF7CE50BC0A9
:1027500006E221EE42EE66EF7CE505C008E221E0EC
:1027600045EE6AED7CE50E94FC1280E008C0FC01A9
:102770008281882319F010922B0201C081E00F9111
:102780000895909389018093880108959093310270
:10279000809330020895E0913002F0913102309739
:1027A00021F00190F081E02D099480E00895E091FE
:1027B0003002F0913102309721F00280F381E02D58
:1027C0000994089520912E0230912F02281739077D
:1027D00071F090932F0280932E02E0913002F091DD
:1027E0003102309721F00680F781E02D0994089599
:1027F00020912C0230912D022817390771F0909307
:102800002D0280932C02E0913002F091310230973A
:1028100021F00084F185E02D09940895FC013296A1
:1028200097E080E0915029F021912223D9F38F5F26
:10283000F9CF0895662349F0FC013296089621915C
:10284000621729F0E817F907D1F780E0089581E0D1
:1028500008959C01FC0132969FEF80E0419146175C
:1028600089F09F3F19F4411101C0982F8F5F863086
:10287000A9F79F3F39F0F901E90FF11D97FDFA958E
:102880006283089508959C012A5F3F4FFC014281B5
:10289000461301C01282019682179307B9F7089573
:1028A0000C9429140C944314029626E0FC01119216
:1028B0002A95E9F7089508950C945B1483E08093BA
:1028C00032020C945C14811102C081E001C082E0EC
:1028D000809332020C945C140C94631481E0809316
:1028E00032020C945C140C946E1408950C947514BC
:1028F0000C9476140C9475140C9475140C94751433
:10290000CF930E947C140E94E4100E947A14C0E0CD
:102910008C2F0E940E10892B29F4CF5FC530C1F790
:1029200080E001C081E0CF91089508951F920F9239
:102930000FB60F9211248F939F93AF93BF93809103
:102940003302811113C08091570290915802A091D7
:102950005902B0915A024196A11DB11D80935702B0
:1029600090935802A0935902B0935A02BF91AF912D
:102970009F918F910F900FBE0F901F90189580918F
:102980005F02843031F10E9467021092330220E42A
:1029900088E190E00FB6F894A895809360000FBE90
:1029A0002093600083B7817F846083BF83B7816099
:1029B00083BF7894889583B78E7F83BF0FB6F894D2
:1029C000A8958091600088618093600010926000FB
:1029D0000FBE08950E9410060C946B0282E084BD25
:1029E00093E095BD9AEF97BD80936E0008952FB741
:1029F000F8948091570290915802A0915902B09199
:102A00005A022FBF08952FB7F89460915702709122
:102A100058028091590290915A022FBF08959C014B
:102A20004FB7F8948091570290915802A0915902A3
:102A3000B0915A024FBF821B930B089578941F9256
:102A40000F920FB60F9211248F939F93AF93BF9362
:102A50008091570290915802A0915902B0915A0268
:102A60000196A11DB11D8093570290935802A09327
:102A70005902B0935A02BF91AF919F918F910F90DD
:102A80000FBE0F901F90189581E08093E00080E2C8
:102A90008093D8001092C9008FE19EE40197F1F76E
:102AA00000C0000087E090EBDC0180936802909307
:102AB0006902A0936A02B0936B029CE088E10FB6B2
:102AC000F894A895809360000FBE90936000FFCFAC
:102AD00080913F0208950895CF93DF9321E02093E2
:102AE000E9002FEF3091E800215035FD06C035EDAB
:102AF0003A95F1F700002111F5CF2091E80025FF6C
:102B000014C0EC0140E050E068E070E00E947817EB
:102B10008091E8008E778093E80088E0FE01A7E3CB
:102B2000B2E001900D928A95E1F7DF91CF9108957F
:102B300080933402709336026093350280915F0275
:102B4000843001F582E08093E9008FEF9091E800F6
:102B5000815095FD06C095ED9A95F1F70000811121
:102B6000F5CF8091E80085FF0DC040E050E063E0C4
:102B700070E084E392E00E9478178091E8008E77FD
:102B80008093E8000895BC0184E00C949815BC0182
:102B900083E00C949815089580915E02811109C01C
:102BA0000E9409190E9466198091E2008460809356
:102BB000E200089510925E0208950C9473146091DF
:102BC0005B0281E0611101C080E00C945E14909181
:102BD0005F0281E0943009F080E060915B020C9428
:102BE000631442E061EC81E00E94821842E261ECF1
:102BF00082E00E94821890915F0281E0943009F097
:102C000080E060915B020C946C14809161028330CF
:102C100009F461C030F4813071F0823009F49AC057
:102C200008958A3009F486C08B3009F46CC089306D
:102C300009F0A8C020C080916002813A09F0A2C0CA
:102C40008091E800877F8093E800809164029091F2
:102C50006502892B21F468E087E392E003C060E01D
:102C600080E090E070E00E94C3178091E8008B77CD
:102C70008093E800089580916002813209F082C05B
:102C80008091640290916502029708F07BC0809168
:102C9000E800877F8093E8008091E80082FD05C00E
:102CA00080915F028111F8CF6DC02091F300809177
:102CB000F20090E0922B029731F48091F100813084
:102CC00011F0863021F48091F10080933F028091D1
:102CD000E8008B7753C080916002813A09F052C0BE
:102CE0008091640290916502892B09F04BC080911C
:102CF000E800877F8093E8008091E80080FFFCCFA8
:102D00008091100136C0809160028132D9F58091A6
:102D1000640290916502892BA9F58091E800877F74
:102D20008093E8000E94B71880916202809310019E
:102D30000C94100680916002813221F58091E800A8
:102D4000877F8093E8000E94B71880916302809388
:102D50004002089580916002813AA1F48091E800D8
:102D6000877F8093E8008091E80080FFFCCF80910E
:102D700040028093F1008091E8008E778093E80014
:102D80000C94B718089584B7877F84BF0FB6F89462
:102D9000A895809160008861809360001092600027
:102DA0000FBE90E080E80FB6F89480936100909396
:102DB00061000FBE0C946E140E9409190E946619DE
:102DC000E2EEF0E080818460808378940C94FB1BB9
:102DD00084E091E00C94C61380915F028530A9F4E1
:102DE00080915F02853079F40E94BF1480915D026A
:102DF0008823B1F30E948014882391F30E94621704
:102E00000E941006EDCF0C94EA14089508950C94D6
:102E10000917292F332723303105C9F060F42130F9
:102E2000310581F02230310509F044C08BE390E098
:102E30002AE232E043C021323105E1F0223231058D
:102E400049F138C082E190E025E632E037C09927A9
:102E50008130910549F028F0029761F5E4E0F2E055
:102E600005C0E6E2F2E002C0E6E1F2E0849190E023
:102E70009F0124C06115710541F061307105D1F4E5
:102E800089E090E025E532E019C089E090E02CE38C
:102E900032E014C06115710541F06130710551F4E3
:102EA00082E390E027E732E009C080E490E029EA7D
:102EB00032E004C080E090E020E030E0FA013183AD
:102EC0002083089580E189BD82E189BD09B400FEB7
:102ED000FDCF8091D8008F7D8093D8008091E00055
:102EE00082608093E0008091E00081FDFCCF089536
:102EF000CF92DF92EF92FF920F931F93CF93DF93C6
:102F0000EC018B017A010E94D618811133C0E114C3
:102F1000F10439F0F70180819181081B190BC80F6A
:102F2000D91FC12CD12C0115110519F18091E80090
:102F300085FD16C08091E8008E778093E800E1144B
:102F4000F10449F0F70180819181C80ED91ED18228
:102F5000C08285E00FC00E94D618882321F30AC0E2
:102F600089918093F10001501109FFEFCF1ADF0A18
:102F7000DACF80E0DF91CF911F910F91FF90EF901A
:102F8000DF90CF9008952091660230916702261756
:102F9000370748F06115710539F42091E8002E7764
:102FA0002093E80001C0B901FC0120E06115710522
:102FB00079F180915F028823F1F18530F1F1809100
:102FC000E80083FD3CC08091E80082FD2EC0809126
:102FD000E80080FFEBCF2091F3008091F20090E0B9
:102FE000922B6115710551F08830910538F42191CB
:102FF0002093F100615071090196F3CF21E0089709
:1030000009F020E08091E8008E778093E800CECF31
:103010002111CFCF0AC080915F02882361F08530F3
:1030200061F08091E80083FD0AC08091E80082FF92
:10303000F2CF80E0089582E0089583E0089581E072
:10304000089520916602309167022617370748F0ED
:103050006115710539F42091E8002E772093E8007E
:1030600001C0B901FC0120E06115710591F1809169
:103070005F02882309F440C0853009F43FC0809185
:10308000E80083FD3DC08091E80082FD2FC0809163
:10309000E80080FFE9CF2091F3008091F20090E0FA
:1030A000922B6115710559F08830910540F42491F7
:1030B0002093F1003196615071090196F2CF21E021
:1030C000089709F020E08091E8008E778093E8006F
:1030D000CBCF2111CCCF0AC080915F02882361F051
:1030E000853061F08091E80083FD0AC08091E8009E
:1030F00082FFF2CF80E0089582E0089583E0089592
:1031000081E00895982F973068F59093E90098171B
:1031100039F07091EC002091ED005091F00003C067
:10312000242F762F50E021FD02C09F5FECCF30911D
:10313000EB003E7F3093EB003091ED003D7F30930C
:10314000ED003091EB0031603093EB007093EC00B8
:103150002093ED005093F0002091EE0027FDE5CF85
:1031600080E008958F708093E90081E00895809158
:10317000600287FF11C08091E80082FD05C0809148
:103180005F028111F8CF11C08091E8008B770BC0EE
:1031900080915F02882349F08091E80080FFF8CF9A
:1031A0008091E8008E778093E80008952091E400F4
:1031B0003091E50095E64091EC00842F817040FF4E
:1031C00023C08091E80080FD1DC080915F028823AC
:1031D00099F0853099F08091EB0085FD11C0409108
:1031E000E4005091E5002417350729F3915011F0C0
:1031F0009A01E1CF84E0089582E0089583E0089584
:1032000081E0089580E008954091E80042FFDDCF1D
:1032100008950E9477190E947F19E0EEF0E0808106
:1032200081608083E8EDF0E080818F77808319BC36
:10323000A7EDB0E08C918E7F8C9380818F7E808310
:1032400010925E0208950F931F93CF93DF930E9415
:1032500077190E947F19C8EDD0E088818F77888325
:1032600088818068888388818F7D888319BC1092CB
:103270005F0210925B0210925D0210925C0200EEFF
:1032800010E0F80180818B7F808388818160888352
:1032900042E060E080E00E948218E1EEF0E0808190
:1032A0008E7F8083E2EEF0E0808181608083808188
:1032B00088608083F80180818E7F8083888180612F
:1032C0008883DF91CF911F910F910895E8EDF0E091
:1032D00080818F7E8083E7EDF0E080818160808354
:1032E00084E082BF81E080935E020C942319E8EDB4
:1032F000F0E080818E7F80831092E200089510922A
:10330000DA001092E10008951F920F920FB60F920B
:1033100011242F933F934F935F936F937F938F93DA
:103320009F93AF93BF93EF93FF938091E10082FF50
:103330000BC08091E20082FF07C08091E1008B7F8B
:103340008093E1000E94FA1B8091DA0080FF1FC089
:103350008091D80080FF1BC08091DA008E7F80931F
:10336000DA008091D90080FF0DC080E189BD82E143
:1033700089BD09B400FEFDCF81E080935F020E9409
:10338000CC1505C019BC10925F020E94DA1580911D
:10339000E10080FF19C08091E20080FF15C080919C
:1033A000E2008E7F8093E2008091E2008061809352
:1033B000E2008091D80080628093D80019BC85E03B
:1033C00080935F020E94DF158091E10084FF30C08E
:1033D0008091E20084FF2CC080E189BD82E189BD3B
:1033E00009B400FEFDCF8091D8008F7D8093D80076
:1033F0008091E1008F7E8093E1008091E2008F7EDA
:103400008093E2008091E20081608093E2008091ED
:103410005B02882311F084E007C08091E30087FD00
:1034200002C081E001C083E080935F020E94E71543
:103430008091E10083FF29C08091E20083FF25C0D5
:103440008091E100877F8093E10082E080935F02BA
:1034500010925B028091E1008E7F8093E100809169
:10346000E2008E7F8093E2008091E2008061809391
:10347000E20042E060E080E00E9482188091F0006B
:1034800088608093F0000E94DD15FF91EF91BF915D
:10349000AF919F918F917F916F915F914F913F91EC
:1034A0002F910F900FBE0F901F9018951F920F92A3
:1034B0000FB60F9211242F933F934F935F936F9307
:1034C0007F938F939F93AF93BF93CF93DF93EF93AC
:1034D000FF93C091E900CF708091EC00D82FD1709C
:1034E00080FDD0E81092E9008091F000877F809302
:1034F000F00078940E949A1A1092E9008091F000EE
:1035000088608093F000CD2BCF70C093E900FF91CD
:10351000EF91DF91CF91BF91AF919F918F917F916B
:103520006F915F914F913F912F910F900FBE0F9030
:103530001F9018951F93CF93DF93CDB7DEB7AA974F
:103540000FB6F894DEBF0FBECDBFE0E6F2E080918B
:10355000F100819322E0E836F207C9F70E940516D0
:103560008091E80083FF2EC18091600290916102FA
:10357000492F50E04A30510508F024C1FA01EE59B4
:10358000FF4F0C94161C803821F0823809F01AC1C4
:1035900008C080915C0290915D02992389F082605D
:1035A0000FC0809164028F70873008F00BC1809348
:1035B000E9008091EB0085FB882780F91092E900F3
:1035C0009091E800977F9093E8008093F10010922B
:1035D000F100D1C0282F2D7F09F0F4C0882319F005
:1035E000823061F0EFC080916202813009F0EAC060
:1035F000933009F080E080935D022EC080916202DA
:1036000081112AC0809164028F702FEF280F26301D
:1036100008F0D8C08093E9002091EB0020FF1CC087
:10362000933021F48091EB00806214C09091EB0004
:1036300090619093EB0021E030E0A90102C0440FBB
:10364000551F8A95E2F74093EA001092EA008091B4
:10365000EB0088608093EB001092E9008091E80015
:10366000877F8093E8000E94B718ACC08111AAC080
:10367000109162021F778091E3008078812B809304
:10368000E3008091E800877F8093E8000E94B718EC
:103690008091E80080FFFCCF8091E30080688093F8
:1036A000E300111102C082E001C083E080935F0259
:1036B00089C08058823008F085C080916202909164
:1036C00063028C3D53E0950779F583E08A838AE2B3
:1036D00089834FB7F894DE01139620E03EE051E273
:1036E000E32FF0E050935700E49120FF03C0E295F0
:1036F000EF703F5FEF708E2F90E0EA3010F0C796CA
:1037000001C0C0968D939D932F5F243149F74FBF21
:103710008091E800877F8093E8006AE270E0CE0144
:1037200001960E94C31716C06091640270916502F1
:10373000AE014F5F5F4F0E940717BC01892B09F450
:1037400041C09091E800977F9093E80089819A8129
:103750000E9421188091E8008B778093E80032C0A6
:10376000803881F58091E800877F8093E800809120
:103770005B028093F1008091E8008E7772CF811117
:1037800021C0809162029091630299270297D4F43C
:103790008091E800877F8093E800809162028093A7
:1037A0005B020E94B71880915B02811106C0809174
:1037B000E30087FD02C081E001C084E080935F02E6
:1037C0000E94F1158091E80083FF0AC08091E80013
:1037D000877F8093E8008091EB0080628093EB000C
:1037E000AA960FB6F894DEBF0FBECDBFDF91CF9182
:1037F0001F9108950895CF9380915F028823A1F0CF
:10380000C091E900CF709091EC00892F817090FDFC
:1038100080E8C82B1092E9008091E80083FD0E94A7
:103820009A1ACF70C093E900CF910895EE0FFF1F51
:103830000590F491E02D0994FB01DC0104C08D9109
:103840000190801921F441505040C8F7881B990B12
:103850000895F999FECF92BD81BDF89A992780B558
:103860000895A8E1B0E042E050E00C945D1C262FE2
:10387000F999FECF92BD81BDF89A019700B4021666
:1038800039F01FBA20BD0FB6F894FA9AF99A0FBE14
:1038900008950396272F0E94381C0E94371C252F5D
:1038A0000E94381C242F0C94381C0196272F0E944C
:1038B000381C0C94371CDC01CB01FC01F999FECFBC
:1038C00006C0F2BDE1BDF89A319600B40D924150A8
:0A38D0005040B8F70895F894FFCFB8
:1038DA00C800080268156C15CB15C715C3156B15FA
:1038EA0001E200E900EA00B500B600B700CD0083A6
:1038FA0001CC008A019201940121022302240225AB
:10390A0002260227022A02B300B4006F0070008167
:10391A008283E200E900EA00B500B600B700CD00F4
:10392A008301CC008A01920194012102230224021C
:10393A002502260227022A02B300B4006F00700093
:10394A00818283929190939535F0366667F1F4F50A
:08395A00F6F734979694C600BD
:00000001FF
